S01B00006275696C642F6D69636132646F742F6D61696E2E73726563E3
S11300000C9446000C9463000C9463000C946300FD
S11300100C9463000C9463000C9463000C946300D0
S11300200C9463000C9463000C9463000C946300C0
S11300300C9463000C9463000C9463000C94C10151
S11300400C9463000C9463000C9463000C946300A0
S11300500C9463000C9463000C9463000C94630090
S11300600C9463000C9463000C9463000C94630080
S11300700C9463000C9463000C9463000C94630070
S11300800C9463000C9463000C94630011241FBE51
S1130090CFEFD0E1DEBFCDBF11E0A0E0B1E0E0EEF4
S11300A0F6E000E00BBF02C007900D92A230B1074A
S11300B0D9F711E0A2E0B1E001C01D92A133B1076C
S11300C0E1F70C94B7000C94000026EE80912C010B
S11300D090912D01A0912E01B0912F010097A105BF
S11300E0B10589F080FF0FC080911E0190911F011E
S11300F0A0912001B0912101863E9105A105B10591
S113010014F420911E018FB7F894992720932801A5
S113011021BF109225018FBF0E94AF010895AC0149
S11301208FB7F894282F3327E0912401809124017C
S11301308F5F809324018091240187708093240130
S11301409091240180911801981759F02FBFFF272F
S1130150EE0FFF1FE95FFE4F4083518381E090E083
S11301600895E09324012FBF80E090E00895CFEF3D
S1130170D0E1DEBFCDBF1ABA17BA11BA92E092B974
S113018093B9D29AD09AD19A8B98809161008F7743
S1130190809361001798A79AA69AA59AA49AA39AFD
S11301A0A29AA19AA09A8D9A8F9A8E9ABB98BF9878
S11301B0159AD79AD39A1D9ADF9ADA9A9F5F9C5F11
S11301C09739E8F370E08AE0809304017093240186
S11301D07093180110922C0110922D0110922E018F
S11301E010922F01709325018FEF8093300180933B
S11301F0020170930501872F8D5F8093260196EE8F
S1130200909328018FB7F894282F332787B78E7FD0
S113021087BF87B78D7F87BF80B7886080BF8BE03B
S113022083BF72BF91BF87B7826087BF2FBF8FB76D
S1130230F894992770932A01DA9AD89AD99A8FBF99
S113024081E090E080932B01709327018093230138
S113025028EE33E040E050E0682F872F0E946201CF
S113026078949091180180912401981719F480E0F2
S113027090E01FC08FB7F894282F3327909118016E
S1130280809118018F5F8093180180911801877005
S113029080931801E92FFF27EE0FFF1FE95FFE4F40
S11302A080819181108211822FBFFC01099581E028
S11302B090E08823B1F685B7806285BF88950000F9
S11302C00000CFCFCF93DF93782F882311F46230CF
S11302D01CF080E090E040C020931A0130931B0191
S11302E040931C0150931D01609319018FB7F8943A
S11302F0C82FDD2782B7280F311D411D511D2093C2
S11303001E0130931F0140932001509321018091DD
S11303102C0190912D01A0912E01B0912F018160AB
S113032080932C0190932D01A0932E01B0932F0163
S1130330809128019927AA27BB27281739074A073C
S11303405B0738F42093280121BF709325010E9494
S1130350AF01CFBF81E090E0DF91CF91089580910C
S11303600001882329F481EA92E00E948F0006C0EC
S113037085B7837E85BF85B7806285BF80E090E0C6
S1130380089578941F920F920FB60F9211242F9311
S11303903F934F935F936F937F938F939F93AF9309
S11303A0BF93EF93FF938FB7F894282F332780914F
S11303B00601882369F080912201809329018860D5
S11303C08093220183BF8091170181BF109206019F
S11303D02FBF8DE192E00E948F00FF91EF91BF91BA
S11303E0AF919F918F917F916F915F914F913F91C9
S11303F02F910F900FBE0F901F9018958FB7F89400
S1130400382F20912A0120FF06C08FB7F89499272E
S1130410DA9A2E7F05C08FB7F8949927DA9821606D
S113042020932A018FBF3FBF81E090E008958FBFE2
S113043008958FB7F89499270895CF93DF9381E0B7
S11304408093250180912C0190912D01A0912E0182
S1130450B0912F010097A105B10509F46DC0FD010C
S1130460EC0180FF69C08091280199270196AA2791
S113047097FDA095BA2F20911E0130911F01409144
S1130480200150912101281B390B4A0B5B0B20934F
S11304901E0130931F01409320015093210123300A
S11304A03105410551050CF047C08091190188239D
S11304B0A9F480911A0190911B01A0911C01B091A3
S11304C01D01280F391F4A1F5B1F20931E01309303
S11304D01F01409320015093210114C081E090E05A
S11304E080959095AA2797FDA095BA2F8C239D23DC
S11304F0AE23BF2380932C0190932D01A0932E0152
S1130500B0932F0180913001882319F48FEF8093E9
S11305103001909130019F5F9093300180910501EB
S11305208F5F80930501E92FFF27ED5FFE4F108257
S113053089ED92E00E948F000E946500DF91CF91C7
S1130540089587B799278C7F009719F080E090E091
S11305501AC06F9918C0379B03C088E090E013C09D
S113056087B7992783709070892B59F081B792B718
S1130570891B803118F48CE190E005C088E190E09B
S113058002C080E190E0382F25B7237E8C3121F022
S1130590883111F008C0000080B7992787709070E7
S11305A0892BC9F7237E232B25BF85B7806285BF9E
S11305B00895CF93DF9390910501992319F4C1E035
S11305C0D0E016C080910201882319F48FEF809344
S11305D00201809102018F5F8093020191509093F8
S11305E00501E82FFF27ED5FFE4F8081C82FDD272F
S11305F0CC2309F04BC0209123012223F1F00E9467
S1130600FE0180912B01282F332788EE93E0B90156
S11306100E944903CB01AA2797FDA095BA2F9C01FC
S1130620AD0161E08C2F0E946201809127018F5FF0
S113063080932701C093230129C031E03093230123
S11306409091270180912B01981751F42093270151
S1130650892F830F80932B01883011F430932B0161
S11306600E94FE0180912B01282F332788EE93E00E
S1130670B9010E944903CB01AA2797FDA095BA2F7F
S11306809C01AD0161E080E00E946201DF91CF91A5
S1130690089597FB092E07260AD077FD04D00CD0C5
S11306A006D000201AF4709561957F4F0895F6F7EF
S11306B0909581959F4F0895AA1BBB1B51E107C0DC
S11306C0AA1FBB1FA617B70710F0A61BB70B881FDE
S11306D0991F5A95A9F780959095BC01CD0108956D
S10506E0010013
S9030000FC
